Component: ARM Compiler 5.06 update 5 (build 528) Tool: armlink [4d35e2]

==============================================================================

Section Cross References

    principale.o(moncode) refers to initialisation.o(i.Init_Cible) for Init_Cible
    stm32f10x_rcc.o(i.RCC_GetClocksFreq) refers to stm32f10x_rcc.o(.data) for APBAHBPrescTable
    stm32f10x_rcc.o(i.RCC_WaitForHSEStartUp) refers to stm32f10x_rcc.o(i.RCC_GetFlagStatus) for RCC_GetFlagStatus
    stm32f10x_spi.o(i.I2S_Init) refers to stm32f10x_rcc.o(i.RCC_GetClocksFreq) for RCC_GetClocksFreq
    stm32f10x_spi.o(i.SPI_I2S_DeInit) refers to stm32f10x_rcc.o(i.RCC_APB2PeriphResetCmd) for RCC_APB2PeriphResetCmd
    stm32f10x_spi.o(i.SPI_I2S_DeInit) refers to stm32f10x_rcc.o(i.RCC_APB1PeriphResetCmd) for RCC_APB1PeriphResetCmd
    stm32f10x_tim.o(i.TIM_DeInit) refers to stm32f10x_rcc.o(i.RCC_APB2PeriphResetCmd) for RCC_APB2PeriphResetCmd
    stm32f10x_tim.o(i.TIM_DeInit) refers to stm32f10x_rcc.o(i.RCC_APB1PeriphResetCmd) for RCC_APB1PeriphResetCmd
    stm32f10x_tim.o(i.TIM_ETRClockMode1Config) refers to stm32f10x_tim.o(i.TIM_ETRConfig) for TIM_ETRConfig
    stm32f10x_tim.o(i.TIM_ETRClockMode2Config) refers to stm32f10x_tim.o(i.TIM_ETRConfig) for TIM_ETRConfig
    stm32f10x_tim.o(i.TIM_ICInit) refers to stm32f10x_tim.o(i.TI1_Config) for TI1_Config
    stm32f10x_tim.o(i.TIM_ICInit) refers to stm32f10x_tim.o(i.TIM_SetIC1Prescaler) for TIM_SetIC1Prescaler
    stm32f10x_tim.o(i.TIM_ICInit) refers to stm32f10x_tim.o(i.TI2_Config) for TI2_Config
    stm32f10x_tim.o(i.TIM_ICInit) refers to stm32f10x_tim.o(i.TIM_SetIC2Prescaler) for TIM_SetIC2Prescaler
    stm32f10x_tim.o(i.TIM_ICInit) refers to stm32f10x_tim.o(i.TI3_Config) for TI3_Config
    stm32f10x_tim.o(i.TIM_ICInit) refers to stm32f10x_tim.o(i.TIM_SetIC3Prescaler) for TIM_SetIC3Prescaler
    stm32f10x_tim.o(i.TIM_ICInit) refers to stm32f10x_tim.o(i.TI4_Config) for TI4_Config
    stm32f10x_tim.o(i.TIM_ICInit) refers to stm32f10x_tim.o(i.TIM_SetIC4Prescaler) for TIM_SetIC4Prescaler
    stm32f10x_tim.o(i.TIM_ITRxExternalClockConfig) refers to stm32f10x_tim.o(i.TIM_SelectInputTrigger) for TIM_SelectInputTrigger
    stm32f10x_tim.o(i.TIM_PWMIConfig) refers to stm32f10x_tim.o(i.TI1_Config) for TI1_Config
    stm32f10x_tim.o(i.TIM_PWMIConfig) refers to stm32f10x_tim.o(i.TIM_SetIC1Prescaler) for TIM_SetIC1Prescaler
    stm32f10x_tim.o(i.TIM_PWMIConfig) refers to stm32f10x_tim.o(i.TI2_Config) for TI2_Config
    stm32f10x_tim.o(i.TIM_PWMIConfig) refers to stm32f10x_tim.o(i.TIM_SetIC2Prescaler) for TIM_SetIC2Prescaler
    stm32f10x_tim.o(i.TIM_TIxExternalClockConfig) refers to stm32f10x_tim.o(i.TI2_Config) for TI2_Config
    stm32f10x_tim.o(i.TIM_TIxExternalClockConfig) refers to stm32f10x_tim.o(i.TI1_Config) for TI1_Config
    stm32f10x_tim.o(i.TIM_TIxExternalClockConfig) refers to stm32f10x_tim.o(i.TIM_SelectInputTrigger) for TIM_SelectInputTrigger
    dma_stm32f10x.o(i.DMA1_Channel1_IRQHandler) refers to dma_stm32f10x.o(i.DMA1_Channel1_Event) for DMA1_Channel1_Event
    dma_stm32f10x.o(i.DMA1_Channel2_IRQHandler) refers to dma_stm32f10x.o(i.DMA1_Channel2_Event) for DMA1_Channel2_Event
    dma_stm32f10x.o(i.DMA1_Channel3_IRQHandler) refers to dma_stm32f10x.o(i.DMA1_Channel3_Event) for DMA1_Channel3_Event
    dma_stm32f10x.o(i.DMA1_Channel4_IRQHandler) refers to dma_stm32f10x.o(i.DMA1_Channel4_Event) for DMA1_Channel4_Event
    dma_stm32f10x.o(i.DMA1_Channel5_IRQHandler) refers to dma_stm32f10x.o(i.DMA1_Channel5_Event) for DMA1_Channel5_Event
    dma_stm32f10x.o(i.DMA1_Channel6_IRQHandler) refers to dma_stm32f10x.o(i.DMA1_Channel6_Event) for DMA1_Channel6_Event
    dma_stm32f10x.o(i.DMA1_Channel7_IRQHandler) refers to dma_stm32f10x.o(i.DMA1_Channel7_Event) for DMA1_Channel7_Event
    dma_stm32f10x.o(i.DMA_ChannelInitialize) refers to dma_stm32f10x.o(i.__NVIC_ClearPendingIRQ) for __NVIC_ClearPendingIRQ
    dma_stm32f10x.o(i.DMA_ChannelInitialize) refers to dma_stm32f10x.o(i.__NVIC_EnableIRQ) for __NVIC_EnableIRQ
    dma_stm32f10x.o(i.DMA_ChannelInitialize) refers to dma_stm32f10x.o(.data) for DMA1_Channel
    dma_stm32f10x.o(i.DMA_ChannelUninitialize) refers to dma_stm32f10x.o(i.__NVIC_DisableIRQ) for __NVIC_DisableIRQ
    dma_stm32f10x.o(i.DMA_ChannelUninitialize) refers to dma_stm32f10x.o(.data) for DMA1_Channel
    gpio_stm32f10x.o(i.GPIO_PinConfigure) refers to gpio_stm32f10x.o(i.GPIO_GetPortClockState) for GPIO_GetPortClockState
    gpio_stm32f10x.o(i.GPIO_PinConfigure) refers to gpio_stm32f10x.o(i.GPIO_PortClock) for GPIO_PortClock
    startup_stm32f10x_md.o(RESET) refers to startup_stm32f10x_md.o(STACK) for __initial_sp
    startup_stm32f10x_md.o(RESET) refers to startup_stm32f10x_md.o(.text) for Reset_Handler
    startup_stm32f10x_md.o(RESET) refers to timer_systick_1.o(i.SysTick_Handler) for SysTick_Handler
    startup_stm32f10x_md.o(RESET) refers to dma_stm32f10x.o(i.DMA1_Channel1_IRQHandler) for DMA1_Channel1_IRQHandler
    startup_stm32f10x_md.o(RESET) refers to dma_stm32f10x.o(i.DMA1_Channel2_IRQHandler) for DMA1_Channel2_IRQHandler
    startup_stm32f10x_md.o(RESET) refers to dma_stm32f10x.o(i.DMA1_Channel3_IRQHandler) for DMA1_Channel3_IRQHandler
    startup_stm32f10x_md.o(RESET) refers to dma_stm32f10x.o(i.DMA1_Channel4_IRQHandler) for DMA1_Channel4_IRQHandler
    startup_stm32f10x_md.o(RESET) refers to dma_stm32f10x.o(i.DMA1_Channel5_IRQHandler) for DMA1_Channel5_IRQHandler
    startup_stm32f10x_md.o(RESET) refers to dma_stm32f10x.o(i.DMA1_Channel6_IRQHandler) for DMA1_Channel6_IRQHandler
    startup_stm32f10x_md.o(RESET) refers to dma_stm32f10x.o(i.DMA1_Channel7_IRQHandler) for DMA1_Channel7_IRQHandler
    startup_stm32f10x_md.o(RESET) refers to fonctiontimer.o(i.TIM1_UP_IRQHandler) for TIM1_UP_IRQHandler
    startup_stm32f10x_md.o(RESET) refers to fonctiontimer.o(i.TIM1_CC_IRQHandler) for TIM1_CC_IRQHandler
    startup_stm32f10x_md.o(RESET) refers to fonctiontimer.o(i.TIM2_IRQHandler) for TIM2_IRQHandler
    startup_stm32f10x_md.o(RESET) refers to fonctiontimer.o(i.TIM3_IRQHandler) for TIM3_IRQHandler
    startup_stm32f10x_md.o(RESET) refers to fonctiontimer.o(i.TIM4_IRQHandler) for TIM4_IRQHandler
    startup_stm32f10x_md.o(.text) refers to system_stm32f10x.o(i.SystemInit) for SystemInit
    startup_stm32f10x_md.o(.text) refers to entry.o(.ARM.Collect$$$$00000000) for __main
    system_stm32f10x.o(i.SetSysClock) refers to system_stm32f10x.o(i.SetSysClockTo72) for SetSysClockTo72
    system_stm32f10x.o(i.SystemCoreClockUpdate) refers to system_stm32f10x.o(.data) for SystemCoreClock
    system_stm32f10x.o(i.SystemInit) refers to system_stm32f10x.o(i.SetSysClock) for SetSysClock
    initialisation.o(i.Init_Cible) refers to initialisation.o(i.Init_Port) for Init_Port
    initialisation.o(i.Init_Cible) refers to initialisation.o(i.Init_Dot) for Init_Dot
    initialisation.o(i.Init_Cible) refers to initialisation.o(i.Init_Timer1) for Init_Timer1
    initialisation.o(i.Init_Cible) refers to initialisation.o(i.Init_Timer2_PWM) for Init_Timer2_PWM
    initialisation.o(i.Init_Cible) refers to initialisation.o(i.Init_Timer3_Slave) for Init_Timer3_Slave
    initialisation.o(i.Init_Cible) refers to initialisation.o(i.Init_Timer4) for Init_Timer4
    initialisation.o(i.Init_Cible) refers to spi.o(i.Config_SPI) for Config_SPI
    initialisation.o(i.Init_Cible) refers to foncasm.o(moncode) for Envoie192Boucle
    initialisation.o(i.Init_Cible) refers to pilote_io_1.o(i.Port_IO_Set) for Port_IO_Set
    initialisation.o(i.Init_Cible) refers to pilote_io_1.o(i.Port_IO_Reset) for Port_IO_Reset
    initialisation.o(i.Init_Cible) refers to timer_systick_1.o(i.Systick_Period) for Systick_Period
    initialisation.o(i.Init_Cible) refers to timer_systick_1.o(i.Systick_Prio_IT) for Systick_Prio_IT
    initialisation.o(i.Init_Cible) refers to initialisation.o(.data) for PrtSurImage
    initialisation.o(i.Init_Cible) refers to warning.o(.data) for warning
    initialisation.o(i.Init_Cible) refers to fonctiontimer.o(i.Anim) for Anim
    initialisation.o(i.Init_Dot) refers to pilote_io_1.o(i.Port_IO_Set) for Port_IO_Set
    initialisation.o(i.Init_Dot) refers to pilote_io_1.o(i.Port_IO_Reset) for Port_IO_Reset
    initialisation.o(i.Init_Dot) refers to foncasm.o(moncode) for Envoie96Dot
    initialisation.o(i.Init_Dot) refers to initialisation.o(.data) for CinqDots
    initialisation.o(i.Init_Port) refers to pilote_io_1.o(i.GPIO_Configure) for GPIO_Configure
    initialisation.o(i.Init_Port_SPI) refers to pilote_io_1.o(i.GPIO_Configure) for GPIO_Configure
    initialisation.o(i.Init_Timer1) refers to ffltui.o(.text) for __aeabi_ui2f
    initialisation.o(i.Init_Timer1) refers to f2d.o(.text) for __aeabi_f2d
    initialisation.o(i.Init_Timer1) refers to dmul.o(.text) for __aeabi_dmul
    initialisation.o(i.Init_Timer1) refers to ddiv.o(.text) for __aeabi_ddiv
    initialisation.o(i.Init_Timer1) refers to d2f.o(.text) for __aeabi_d2f
    initialisation.o(i.Init_Timer1) refers to fmul.o(.text) for __aeabi_fmul
    initialisation.o(i.Init_Timer1) refers to cdcmple.o(.text) for __aeabi_cdcmple
    initialisation.o(i.Init_Timer1) refers to cdrcmple.o(.text) for __aeabi_cdrcmple
    initialisation.o(i.Init_Timer1) refers to ffixui.o(.text) for __aeabi_f2uiz
    initialisation.o(i.Init_Timer2_PWM) refers to f2d.o(.text) for __aeabi_f2d
    initialisation.o(i.Init_Timer2_PWM) refers to ddiv.o(.text) for __aeabi_ddiv
    initialisation.o(i.Init_Timer2_PWM) refers to d2f.o(.text) for __aeabi_d2f
    initialisation.o(i.Init_Timer2_PWM) refers to ffltui.o(.text) for __aeabi_ui2f
    initialisation.o(i.Init_Timer2_PWM) refers to fmul.o(.text) for __aeabi_fmul
    initialisation.o(i.Init_Timer2_PWM) refers to ffixui.o(.text) for __aeabi_f2uiz
    initialisation.o(i.Init_Timer2_PWM) refers to fdiv.o(.text) for __aeabi_fdiv
    fonctiontimer.o(i.Anim) refers to fonctiontimer.o(.data) for ImageEnCours
    fonctiontimer.o(i.TIM1_CC_IRQHandler) refers to fonctiontimer.o(.data) for SecteurEnCours
    fonctiontimer.o(i.TIM1_UP_IRQHandler) refers to foncasm.o(moncode) for Envoie192Boucle
    fonctiontimer.o(i.TIM1_UP_IRQHandler) refers to fonctiontimer.o(.data) for VitesseSuffisante
    fonctiontimer.o(i.TIM1_UP_IRQHandler) refers to warning.o(.data) for warning
    fonctiontimer.o(i.TIM1_UP_IRQHandler) refers to initialisation.o(.data) for DataSend
    fonctiontimer.o(i.TIM3_IRQHandler) refers to pilote_io_1.o(i.Port_IO_Set) for Port_IO_Set
    fonctiontimer.o(i.TIM3_IRQHandler) refers to pilote_io_1.o(i.Port_IO_Reset) for Port_IO_Reset
    fonctiontimer.o(i.TIM3_IRQHandler) refers to initialisation.o(.data) for DataSend
    fonctiontimer.o(i.TIM4_IRQHandler) refers to spi.o(i.SendSPI) for SendSPI
    fonctiontimer.o(i.TIM4_IRQHandler) refers to fonctiontimer.o(.data) for SecteurEnCours
    fonctiontimer.o(i.TIM4_IRQHandler) refers to initialisation.o(.data) for PrtSurImage
    spi.o(i.Config_SPI) refers to stm32f10x_spi.o(i.SPI_Init) for SPI_Init
    spi.o(i.Config_SPI) refers to stm32f10x_spi.o(i.SPI_Cmd) for SPI_Cmd
    spi.o(i.Config_SPI) refers to spi.o(.bss) for SPI_InitStructure
    spi.o(i.SendSPI) refers to stm32f10x_spi.o(i.SPI_I2S_GetFlagStatus) for SPI_I2S_GetFlagStatus
    spi.o(i.SendSPI) refers to spi.o(i.SPI_I2S_SendData16) for SPI_I2S_SendData16
    foncasm.o(moncode) refers to initialisation.o(.data) for BarretEnCours
    timer_systick_1.o(i.SysTick_Handler) refers to timer_systick_1.o(.data) for Ptr_Systick
    timer_systick_1.o(i.Systick_Period) refers to fmul.o(.text) for __aeabi_fmul
    timer_systick_1.o(i.Systick_Period) refers to f2d.o(.text) for __aeabi_f2d
    timer_systick_1.o(i.Systick_Period) refers to ddiv.o(.text) for __aeabi_ddiv
    timer_systick_1.o(i.Systick_Period) refers to d2f.o(.text) for __aeabi_d2f
    timer_systick_1.o(i.Systick_Period) refers to ffixui.o(.text) for __aeabi_f2uiz
    timer_systick_1.o(i.Systick_Period) refers to ffltui.o(.text) for __aeabi_ui2f
    timer_systick_1.o(i.Systick_Period) refers to fdiv.o(.text) for __aeabi_fdiv
    timer_systick_1.o(i.Systick_Period) refers to dmul.o(.text) for __aeabi_dmul
    timer_systick_1.o(i.Systick_Period) refers to cdrcmple.o(.text) for __aeabi_cdrcmple
    timer_systick_1.o(i.Systick_Prio_IT) refers to timer_systick_1.o(.data) for Ptr_Systick
    entry.o(.ARM.Collect$$$$00000000) refers (Special) to entry10a.o(.ARM.Collect$$$$0000000D) for __rt_final_cpp
    entry.o(.ARM.Collect$$$$00000000) refers (Special) to entry11a.o(.ARM.Collect$$$$0000000F) for __rt_final_exit
    entry.o(.ARM.Collect$$$$00000000) refers (Special) to entry7b.o(.ARM.Collect$$$$00000008) for _main_clock
    entry.o(.ARM.Collect$$$$00000000) refers (Special) to entry8b.o(.ARM.Collect$$$$0000000A) for _main_cpp_init
    entry.o(.ARM.Collect$$$$00000000) refers (Special) to entry9a.o(.ARM.Collect$$$$0000000B) for _main_init
    entry.o(.ARM.Collect$$$$00000000) refers (Special) to entry5.o(.ARM.Collect$$$$00000004) for _main_scatterload
    entry.o(.ARM.Collect$$$$00000000) refers (Special) to entry2.o(.ARM.Collect$$$$00000001) for _main_stk
    fmul.o(.text) refers (Special) to iusefp.o(.text) for __I$use$fp
    fdiv.o(.text) refers (Special) to iusefp.o(.text) for __I$use$fp
    fdiv.o(.text) refers to fepilogue.o(.text) for _float_round
    dmul.o(.text) refers (Special) to iusefp.o(.text) for __I$use$fp
    dmul.o(.text) refers to depilogue.o(.text) for _double_epilogue
    ddiv.o(.text) refers (Special) to iusefp.o(.text) for __I$use$fp
    ddiv.o(.text) refers to depilogue.o(.text) for _double_round
    ffltui.o(.text) refers (Special) to iusefp.o(.text) for __I$use$fp
    ffltui.o(.text) refers to fepilogue.o(.text) for _float_epilogue
    ffixui.o(.text) refers (Special) to iusefp.o(.text) for __I$use$fp
    f2d.o(.text) refers (Special) to iusefp.o(.text) for __I$use$fp
    cdcmple.o(.text) refers (Special) to iusefp.o(.text) for __I$use$fp
    cdrcmple.o(.text) refers (Special) to iusefp.o(.text) for __I$use$fp
    d2f.o(.text) refers (Special) to iusefp.o(.text) for __I$use$fp
    d2f.o(.text) refers to fepilogue.o(.text) for _float_round
    entry2.o(.ARM.Collect$$$$00000001) refers to entry2.o(.ARM.Collect$$$$00002712) for __lit__00000000
    entry2.o(.ARM.Collect$$$$00002712) refers to startup_stm32f10x_md.o(STACK) for __initial_sp
    entry2.o(__vectab_stack_and_reset_area) refers to startup_stm32f10x_md.o(STACK) for __initial_sp
    entry2.o(__vectab_stack_and_reset_area) refers to entry.o(.ARM.Collect$$$$00000000) for __main
    entry5.o(.ARM.Collect$$$$00000004) refers to init.o(.text) for __scatterload
    entry9a.o(.ARM.Collect$$$$0000000B) refers to principale.o(moncode) for main
    entry9b.o(.ARM.Collect$$$$0000000C) refers to principale.o(moncode) for main
    depilogue.o(.text) refers to llshl.o(.text) for __aeabi_llsl
    depilogue.o(.text) refers to llushr.o(.text) for __aeabi_llsr
    init.o(.text) refers to entry5.o(.ARM.Collect$$$$00000004) for __main_after_scatterload


==============================================================================

Removing Unused input sections from the image.

    Removing principale.o(mesdonnees), (0 bytes).
    Removing fonctionetape.o(MesDonnees), (0 bytes).
    Removing fonctionetape.o(moncode), (0 bytes).
    Removing misc.o(.rev16_text), (4 bytes).
    Removing misc.o(.revsh_text), (4 bytes).
    Removing misc.o(.rrx_text), (6 bytes).
    Removing misc.o(i.NVIC_Init), (112 bytes).
    Removing misc.o(i.NVIC_PriorityGroupConfig), (20 bytes).
    Removing misc.o(i.NVIC_SetVectorTable), (20 bytes).
    Removing misc.o(i.NVIC_SystemLPConfig), (32 bytes).
    Removing misc.o(i.SysTick_CLKSourceConfig), (40 bytes).
    Removing stm32f10x_rcc.o(.rev16_text), (4 bytes).
    Removing stm32f10x_rcc.o(.revsh_text), (4 bytes).
    Removing stm32f10x_rcc.o(.rrx_text), (6 bytes).
    Removing stm32f10x_rcc.o(i.RCC_ADCCLKConfig), (24 bytes).
    Removing stm32f10x_rcc.o(i.RCC_AHBPeriphClockCmd), (32 bytes).
    Removing stm32f10x_rcc.o(i.RCC_APB1PeriphClockCmd), (32 bytes).
    Removing stm32f10x_rcc.o(i.RCC_APB1PeriphResetCmd), (32 bytes).
    Removing stm32f10x_rcc.o(i.RCC_APB2PeriphClockCmd), (32 bytes).
    Removing stm32f10x_rcc.o(i.RCC_APB2PeriphResetCmd), (32 bytes).
    Removing stm32f10x_rcc.o(i.RCC_AdjustHSICalibrationValue), (24 bytes).
    Removing stm32f10x_rcc.o(i.RCC_BackupResetCmd), (12 bytes).
    Removing stm32f10x_rcc.o(i.RCC_ClearFlag), (20 bytes).
    Removing stm32f10x_rcc.o(i.RCC_ClearITPendingBit), (12 bytes).
    Removing stm32f10x_rcc.o(i.RCC_ClockSecuritySystemCmd), (12 bytes).
    Removing stm32f10x_rcc.o(i.RCC_DeInit), (76 bytes).
    Removing stm32f10x_rcc.o(i.RCC_GetClocksFreq), (212 bytes).
    Removing stm32f10x_rcc.o(i.RCC_GetFlagStatus), (60 bytes).
    Removing stm32f10x_rcc.o(i.RCC_GetITStatus), (24 bytes).
    Removing stm32f10x_rcc.o(i.RCC_GetSYSCLKSource), (16 bytes).
    Removing stm32f10x_rcc.o(i.RCC_HCLKConfig), (24 bytes).
    Removing stm32f10x_rcc.o(i.RCC_HSEConfig), (76 bytes).
    Removing stm32f10x_rcc.o(i.RCC_HSICmd), (12 bytes).
    Removing stm32f10x_rcc.o(i.RCC_ITConfig), (32 bytes).
    Removing stm32f10x_rcc.o(i.RCC_LSEConfig), (52 bytes).
    Removing stm32f10x_rcc.o(i.RCC_LSICmd), (12 bytes).
    Removing stm32f10x_rcc.o(i.RCC_MCOConfig), (12 bytes).
    Removing stm32f10x_rcc.o(i.RCC_PCLK1Config), (24 bytes).
    Removing stm32f10x_rcc.o(i.RCC_PCLK2Config), (24 bytes).
    Removing stm32f10x_rcc.o(i.RCC_PLLCmd), (12 bytes).
    Removing stm32f10x_rcc.o(i.RCC_PLLConfig), (28 bytes).
    Removing stm32f10x_rcc.o(i.RCC_RTCCLKCmd), (12 bytes).
    Removing stm32f10x_rcc.o(i.RCC_RTCCLKConfig), (16 bytes).
    Removing stm32f10x_rcc.o(i.RCC_SYSCLKConfig), (24 bytes).
    Removing stm32f10x_rcc.o(i.RCC_USBCLKConfig), (12 bytes).
    Removing stm32f10x_rcc.o(i.RCC_WaitForHSEStartUp), (56 bytes).
    Removing stm32f10x_rcc.o(.data), (20 bytes).
    Removing stm32f10x_spi.o(.rev16_text), (4 bytes).
    Removing stm32f10x_spi.o(.revsh_text), (4 bytes).
    Removing stm32f10x_spi.o(.rrx_text), (6 bytes).
    Removing stm32f10x_spi.o(i.I2S_Cmd), (24 bytes).
    Removing stm32f10x_spi.o(i.I2S_Init), (232 bytes).
    Removing stm32f10x_spi.o(i.I2S_StructInit), (20 bytes).
    Removing stm32f10x_spi.o(i.SPI_BiDirectionalLineConfig), (28 bytes).
    Removing stm32f10x_spi.o(i.SPI_CalculateCRC), (24 bytes).
    Removing stm32f10x_spi.o(i.SPI_DataSizeConfig), (18 bytes).
    Removing stm32f10x_spi.o(i.SPI_GetCRC), (16 bytes).
    Removing stm32f10x_spi.o(i.SPI_GetCRCPolynomial), (6 bytes).
    Removing stm32f10x_spi.o(i.SPI_I2S_ClearFlag), (6 bytes).
    Removing stm32f10x_spi.o(i.SPI_I2S_ClearITPendingBit), (20 bytes).
    Removing stm32f10x_spi.o(i.SPI_I2S_DMACmd), (18 bytes).
    Removing stm32f10x_spi.o(i.SPI_I2S_DeInit), (88 bytes).
    Removing stm32f10x_spi.o(i.SPI_I2S_GetITStatus), (52 bytes).
    Removing stm32f10x_spi.o(i.SPI_I2S_ITConfig), (32 bytes).
    Removing stm32f10x_spi.o(i.SPI_I2S_ReceiveData), (6 bytes).
    Removing stm32f10x_spi.o(i.SPI_I2S_SendData), (4 bytes).
    Removing stm32f10x_spi.o(i.SPI_NSSInternalSoftwareConfig), (30 bytes).
    Removing stm32f10x_spi.o(i.SPI_SSOutputCmd), (24 bytes).
    Removing stm32f10x_spi.o(i.SPI_StructInit), (24 bytes).
    Removing stm32f10x_spi.o(i.SPI_TransmitCRC), (10 bytes).
    Removing stm32f10x_tim.o(.rev16_text), (4 bytes).
    Removing stm32f10x_tim.o(.revsh_text), (4 bytes).
    Removing stm32f10x_tim.o(.rrx_text), (6 bytes).
    Removing stm32f10x_tim.o(i.TI1_Config), (128 bytes).
    Removing stm32f10x_tim.o(i.TI2_Config), (152 bytes).
    Removing stm32f10x_tim.o(i.TI3_Config), (144 bytes).
    Removing stm32f10x_tim.o(i.TI4_Config), (152 bytes).
    Removing stm32f10x_tim.o(i.TIM_ARRPreloadConfig), (24 bytes).
    Removing stm32f10x_tim.o(i.TIM_BDTRConfig), (32 bytes).
    Removing stm32f10x_tim.o(i.TIM_BDTRStructInit), (18 bytes).
    Removing stm32f10x_tim.o(i.TIM_CCPreloadControl), (24 bytes).
    Removing stm32f10x_tim.o(i.TIM_CCxCmd), (30 bytes).
    Removing stm32f10x_tim.o(i.TIM_CCxNCmd), (30 bytes).
    Removing stm32f10x_tim.o(i.TIM_ClearFlag), (6 bytes).
    Removing stm32f10x_tim.o(i.TIM_ClearITPendingBit), (6 bytes).
    Removing stm32f10x_tim.o(i.TIM_ClearOC1Ref), (18 bytes).
    Removing stm32f10x_tim.o(i.TIM_ClearOC2Ref), (24 bytes).
    Removing stm32f10x_tim.o(i.TIM_ClearOC3Ref), (18 bytes).
    Removing stm32f10x_tim.o(i.TIM_ClearOC4Ref), (24 bytes).
    Removing stm32f10x_tim.o(i.TIM_Cmd), (24 bytes).
    Removing stm32f10x_tim.o(i.TIM_CounterModeConfig), (18 bytes).
    Removing stm32f10x_tim.o(i.TIM_CtrlPWMOutputs), (30 bytes).
    Removing stm32f10x_tim.o(i.TIM_DMACmd), (18 bytes).
    Removing stm32f10x_tim.o(i.TIM_DMAConfig), (10 bytes).
    Removing stm32f10x_tim.o(i.TIM_DeInit), (488 bytes).
    Removing stm32f10x_tim.o(i.TIM_ETRClockMode1Config), (54 bytes).
    Removing stm32f10x_tim.o(i.TIM_ETRClockMode2Config), (32 bytes).
    Removing stm32f10x_tim.o(i.TIM_ETRConfig), (28 bytes).
    Removing stm32f10x_tim.o(i.TIM_EncoderInterfaceConfig), (66 bytes).
    Removing stm32f10x_tim.o(i.TIM_ForcedOC1Config), (18 bytes).
    Removing stm32f10x_tim.o(i.TIM_ForcedOC2Config), (26 bytes).
    Removing stm32f10x_tim.o(i.TIM_ForcedOC3Config), (18 bytes).
    Removing stm32f10x_tim.o(i.TIM_ForcedOC4Config), (26 bytes).
    Removing stm32f10x_tim.o(i.TIM_GenerateEvent), (4 bytes).
    Removing stm32f10x_tim.o(i.TIM_GetCapture1), (6 bytes).
    Removing stm32f10x_tim.o(i.TIM_GetCapture2), (6 bytes).
    Removing stm32f10x_tim.o(i.TIM_GetCapture3), (6 bytes).
    Removing stm32f10x_tim.o(i.TIM_GetCapture4), (8 bytes).
    Removing stm32f10x_tim.o(i.TIM_GetCounter), (6 bytes).
    Removing stm32f10x_tim.o(i.TIM_GetFlagStatus), (18 bytes).
    Removing stm32f10x_tim.o(i.TIM_GetITStatus), (34 bytes).
    Removing stm32f10x_tim.o(i.TIM_GetPrescaler), (6 bytes).
    Removing stm32f10x_tim.o(i.TIM_ICInit), (172 bytes).
    Removing stm32f10x_tim.o(i.TIM_ICStructInit), (18 bytes).
    Removing stm32f10x_tim.o(i.TIM_ITConfig), (18 bytes).
    Removing stm32f10x_tim.o(i.TIM_ITRxExternalClockConfig), (24 bytes).
    Removing stm32f10x_tim.o(i.TIM_InternalClockConfig), (12 bytes).
    Removing stm32f10x_tim.o(i.TIM_OC1FastConfig), (18 bytes).
    Removing stm32f10x_tim.o(i.TIM_OC1Init), (152 bytes).
    Removing stm32f10x_tim.o(i.TIM_OC1NPolarityConfig), (18 bytes).
    Removing stm32f10x_tim.o(i.TIM_OC1PolarityConfig), (18 bytes).
    Removing stm32f10x_tim.o(i.TIM_OC1PreloadConfig), (18 bytes).
    Removing stm32f10x_tim.o(i.TIM_OC2FastConfig), (26 bytes).
    Removing stm32f10x_tim.o(i.TIM_OC2Init), (164 bytes).
    Removing stm32f10x_tim.o(i.TIM_OC2NPolarityConfig), (26 bytes).
    Removing stm32f10x_tim.o(i.TIM_OC2PolarityConfig), (26 bytes).
    Removing stm32f10x_tim.o(i.TIM_OC2PreloadConfig), (26 bytes).
    Removing stm32f10x_tim.o(i.TIM_OC3FastConfig), (18 bytes).
    Removing stm32f10x_tim.o(i.TIM_OC3Init), (160 bytes).
    Removing stm32f10x_tim.o(i.TIM_OC3NPolarityConfig), (26 bytes).
    Removing stm32f10x_tim.o(i.TIM_OC3PolarityConfig), (26 bytes).
    Removing stm32f10x_tim.o(i.TIM_OC3PreloadConfig), (18 bytes).
    Removing stm32f10x_tim.o(i.TIM_OC4FastConfig), (26 bytes).
    Removing stm32f10x_tim.o(i.TIM_OC4Init), (124 bytes).
    Removing stm32f10x_tim.o(i.TIM_OC4PolarityConfig), (26 bytes).
    Removing stm32f10x_tim.o(i.TIM_OC4PreloadConfig), (26 bytes).
    Removing stm32f10x_tim.o(i.TIM_OCStructInit), (20 bytes).
    Removing stm32f10x_tim.o(i.TIM_PWMIConfig), (124 bytes).
    Removing stm32f10x_tim.o(i.TIM_PrescalerConfig), (6 bytes).
    Removing stm32f10x_tim.o(i.TIM_SelectCCDMA), (24 bytes).
    Removing stm32f10x_tim.o(i.TIM_SelectCOM), (24 bytes).
    Removing stm32f10x_tim.o(i.TIM_SelectHallSensor), (24 bytes).
    Removing stm32f10x_tim.o(i.TIM_SelectInputTrigger), (18 bytes).
    Removing stm32f10x_tim.o(i.TIM_SelectMasterSlaveMode), (18 bytes).
    Removing stm32f10x_tim.o(i.TIM_SelectOCxM), (82 bytes).
    Removing stm32f10x_tim.o(i.TIM_SelectOnePulseMode), (18 bytes).
    Removing stm32f10x_tim.o(i.TIM_SelectOutputTrigger), (18 bytes).
    Removing stm32f10x_tim.o(i.TIM_SelectSlaveMode), (18 bytes).
    Removing stm32f10x_tim.o(i.TIM_SetAutoreload), (4 bytes).
    Removing stm32f10x_tim.o(i.TIM_SetClockDivision), (18 bytes).
    Removing stm32f10x_tim.o(i.TIM_SetCompare1), (4 bytes).
    Removing stm32f10x_tim.o(i.TIM_SetCompare2), (4 bytes).
    Removing stm32f10x_tim.o(i.TIM_SetCompare3), (4 bytes).
    Removing stm32f10x_tim.o(i.TIM_SetCompare4), (6 bytes).
    Removing stm32f10x_tim.o(i.TIM_SetCounter), (4 bytes).
    Removing stm32f10x_tim.o(i.TIM_SetIC1Prescaler), (18 bytes).
    Removing stm32f10x_tim.o(i.TIM_SetIC2Prescaler), (26 bytes).
    Removing stm32f10x_tim.o(i.TIM_SetIC3Prescaler), (18 bytes).
    Removing stm32f10x_tim.o(i.TIM_SetIC4Prescaler), (26 bytes).
    Removing stm32f10x_tim.o(i.TIM_TIxExternalClockConfig), (62 bytes).
    Removing stm32f10x_tim.o(i.TIM_TimeBaseInit), (164 bytes).
    Removing stm32f10x_tim.o(i.TIM_TimeBaseStructInit), (18 bytes).
    Removing stm32f10x_tim.o(i.TIM_UpdateDisableConfig), (24 bytes).
    Removing stm32f10x_tim.o(i.TIM_UpdateRequestConfig), (24 bytes).
    Removing dma_stm32f10x.o(.rev16_text), (4 bytes).
    Removing dma_stm32f10x.o(.revsh_text), (4 bytes).
    Removing dma_stm32f10x.o(.rrx_text), (6 bytes).
    Removing dma_stm32f10x.o(i.DMA_ChannelInitialize), (256 bytes).
    Removing dma_stm32f10x.o(i.DMA_ChannelUninitialize), (188 bytes).
    Removing dma_stm32f10x.o(i.__NVIC_ClearPendingIRQ), (28 bytes).
    Removing dma_stm32f10x.o(i.__NVIC_DisableIRQ), (60 bytes).
    Removing dma_stm32f10x.o(i.__NVIC_EnableIRQ), (26 bytes).
    Removing dma_stm32f10x.o(.data), (1 bytes).
    Removing gpio_stm32f10x.o(.rev16_text), (4 bytes).
    Removing gpio_stm32f10x.o(.revsh_text), (4 bytes).
    Removing gpio_stm32f10x.o(.rrx_text), (6 bytes).
    Removing gpio_stm32f10x.o(i.GPIO_AFConfigure), (156 bytes).
    Removing gpio_stm32f10x.o(i.GPIO_GetPortClockState), (152 bytes).
    Removing gpio_stm32f10x.o(i.GPIO_PinConfigure), (120 bytes).
    Removing gpio_stm32f10x.o(i.GPIO_PortClock), (316 bytes).
    Removing startup_stm32f10x_md.o(HEAP), (512 bytes).
    Removing system_stm32f10x.o(.rev16_text), (4 bytes).
    Removing system_stm32f10x.o(.revsh_text), (4 bytes).
    Removing system_stm32f10x.o(.rrx_text), (6 bytes).
    Removing system_stm32f10x.o(i.SystemCoreClockUpdate), (164 bytes).
    Removing system_stm32f10x.o(.data), (20 bytes).
    Removing initialisation.o(.rev16_text), (4 bytes).
    Removing initialisation.o(.revsh_text), (4 bytes).
    Removing initialisation.o(.rrx_text), (6 bytes).
    Removing initialisation.o(i.Init_Port_SPI), (76 bytes).
    Removing fonctiontimer.o(.rev16_text), (4 bytes).
    Removing fonctiontimer.o(.revsh_text), (4 bytes).
    Removing fonctiontimer.o(.rrx_text), (6 bytes).
    Removing fonctiontimer.o(i.Run_Timer1), (20 bytes).
    Removing fonctiontimer.o(i.Run_Timer2), (18 bytes).
    Removing fonctiontimer.o(i.Run_Timer3), (20 bytes).
    Removing fonctiontimer.o(i.Run_Timer4), (20 bytes).
    Removing fonctiontimer.o(i.Stop_Timer1), (20 bytes).
    Removing fonctiontimer.o(i.Stop_Timer2), (18 bytes).
    Removing fonctiontimer.o(i.Stop_Timer3), (20 bytes).
    Removing fonctiontimer.o(i.Stop_Timer4), (20 bytes).
    Removing spi.o(.rev16_text), (4 bytes).
    Removing spi.o(.revsh_text), (4 bytes).
    Removing spi.o(.rrx_text), (6 bytes).
    Removing foncasm.o(muu), (0 bytes).
    Removing pilote_io_1.o(.rev16_text), (4 bytes).
    Removing pilote_io_1.o(.revsh_text), (4 bytes).
    Removing pilote_io_1.o(.rrx_text), (6 bytes).
    Removing pilote_io_1.o(i.Port_IO_Blink), (16 bytes).
    Removing pilote_io_1.o(i.Port_IO_Init_Input), (74 bytes).
    Removing pilote_io_1.o(i.Port_IO_Init_Input_Analog), (46 bytes).
    Removing pilote_io_1.o(i.Port_IO_Init_Output), (74 bytes).
    Removing pilote_io_1.o(i.Port_IO_Read), (12 bytes).
    Removing timer_systick_1.o(.rev16_text), (4 bytes).
    Removing timer_systick_1.o(.revsh_text), (4 bytes).
    Removing timer_systick_1.o(.rrx_text), (6 bytes).

216 unused section(s) (total 8411 bytes) removed from the image.

==============================================================================

Image Symbol Table

    Local Symbols

    Symbol Name                              Value     Ov Type        Size  Object(Section)

    ../clib/microlib/init/entry.s            0x00000000   Number         0  entry7a.o ABSOLUTE
    ../clib/microlib/init/entry.s            0x00000000   Number         0  entry8b.o ABSOLUTE
    ../clib/microlib/init/entry.s            0x00000000   Number         0  entry9a.o ABSOLUTE
    ../clib/microlib/init/entry.s            0x00000000   Number         0  entry11b.o ABSOLUTE
    ../clib/microlib/init/entry.s            0x00000000   Number         0  entry10b.o ABSOLUTE
    ../clib/microlib/init/entry.s            0x00000000   Number         0  entry10a.o ABSOLUTE
    ../clib/microlib/init/entry.s            0x00000000   Number         0  entry7b.o ABSOLUTE
    ../clib/microlib/init/entry.s            0x00000000   Number         0  entry11a.o ABSOLUTE
    ../clib/microlib/init/entry.s            0x00000000   Number         0  entry9b.o ABSOLUTE
    ../clib/microlib/init/entry.s            0x00000000   Number         0  entry8a.o ABSOLUTE
    ../clib/microlib/init/entry.s            0x00000000   Number         0  entry.o ABSOLUTE
    ../clib/microlib/init/entry.s            0x00000000   Number         0  entry5.o ABSOLUTE
    ../clib/microlib/init/entry.s            0x00000000   Number         0  entry2.o ABSOLUTE
    ../clib/microlib/longlong.c              0x00000000   Number         0  llushr.o ABSOLUTE
    ../clib/microlib/longlong.c              0x00000000   Number         0  llshl.o ABSOLUTE
    ../clib/microlib/stubs.s                 0x00000000   Number         0  iusefp.o ABSOLUTE
    ../fplib/microlib/d2f.c                  0x00000000   Number         0  d2f.o ABSOLUTE
    ../fplib/microlib/f2d.c                  0x00000000   Number         0  f2d.o ABSOLUTE
    ../fplib/microlib/fpdiv.c                0x00000000   Number         0  ddiv.o ABSOLUTE
    ../fplib/microlib/fpdiv.c                0x00000000   Number         0  fdiv.o ABSOLUTE
    ../fplib/microlib/fpepilogue.c           0x00000000   Number         0  depilogue.o ABSOLUTE
    ../fplib/microlib/fpepilogue.c           0x00000000   Number         0  fepilogue.o ABSOLUTE
    ../fplib/microlib/fpfix.c                0x00000000   Number         0  ffixui.o ABSOLUTE
    ../fplib/microlib/fpflt.c                0x00000000   Number         0  ffltui.o ABSOLUTE
    ../fplib/microlib/fpmul.c                0x00000000   Number         0  fmul.o ABSOLUTE
    ../fplib/microlib/fpmul.c                0x00000000   Number         0  dmul.o ABSOLUTE
    ..\\pilotes\\Sources\\Timer_Systick.c    0x00000000   Number         0  timer_systick_1.o ABSOLUTE
    ..\\pilotes\\Sources\\pilote_IO.c        0x00000000   Number         0  pilote_io_1.o ABSOLUTE
    ..\pilotes\Sources\Timer_Systick.c       0x00000000   Number         0  timer_systick_1.o ABSOLUTE
    ..\pilotes\Sources\pilote_IO.c           0x00000000   Number         0  pilote_io_1.o ABSOLUTE
    C:\Keil_v5\ARM\PACK\Keil\STM32F1xx_DFP\2.2.0\Device\StdPeriph_Driver\src\misc.c 0x00000000   Number         0  misc.o ABSOLUTE
    C:\Keil_v5\ARM\PACK\Keil\STM32F1xx_DFP\2.2.0\Device\StdPeriph_Driver\src\stm32f10x_rcc.c 0x00000000   Number         0  stm32f10x_rcc.o ABSOLUTE
    C:\Keil_v5\ARM\PACK\Keil\STM32F1xx_DFP\2.2.0\Device\StdPeriph_Driver\src\stm32f10x_spi.c 0x00000000   Number         0  stm32f10x_spi.o ABSOLUTE
    C:\Keil_v5\ARM\PACK\Keil\STM32F1xx_DFP\2.2.0\Device\StdPeriph_Driver\src\stm32f10x_tim.c 0x00000000   Number         0  stm32f10x_tim.o ABSOLUTE
    C:\Keil_v5\ARM\PACK\Keil\STM32F1xx_DFP\2.2.0\RTE_Driver\DMA_STM32F10x.c 0x00000000   Number         0  dma_stm32f10x.o ABSOLUTE
    C:\Keil_v5\ARM\PACK\Keil\STM32F1xx_DFP\2.2.0\RTE_Driver\GPIO_STM32F10x.c 0x00000000   Number         0  gpio_stm32f10x.o ABSOLUTE
    C:\\Keil_v5\\ARM\\PACK\\Keil\\STM32F1xx_DFP\\2.2.0\\Device\\StdPeriph_Driver\\src\\misc.c 0x00000000   Number         0  misc.o ABSOLUTE
    C:\\Keil_v5\\ARM\\PACK\\Keil\\STM32F1xx_DFP\\2.2.0\\Device\\StdPeriph_Driver\\src\\stm32f10x_rcc.c 0x00000000   Number         0  stm32f10x_rcc.o ABSOLUTE
    C:\\Keil_v5\\ARM\\PACK\\Keil\\STM32F1xx_DFP\\2.2.0\\Device\\StdPeriph_Driver\\src\\stm32f10x_spi.c 0x00000000   Number         0  stm32f10x_spi.o ABSOLUTE
    C:\\Keil_v5\\ARM\\PACK\\Keil\\STM32F1xx_DFP\\2.2.0\\Device\\StdPeriph_Driver\\src\\stm32f10x_tim.c 0x00000000   Number         0  stm32f10x_tim.o ABSOLUTE
    C:\\Keil_v5\\ARM\\PACK\\Keil\\STM32F1xx_DFP\\2.2.0\\RTE_Driver\\DMA_STM32F10x.c 0x00000000   Number         0  dma_stm32f10x.o ABSOLUTE
    C:\\Keil_v5\\ARM\\PACK\\Keil\\STM32F1xx_DFP\\2.2.0\\RTE_Driver\\GPIO_STM32F10x.c 0x00000000   Number         0  gpio_stm32f10x.o ABSOLUTE
    FoncAsm.asm                              0x00000000   Number         0  foncasm.o ABSOLUTE
    FonctionEtape.asm                        0x00000000   Number         0  fonctionetape.o ABSOLUTE
    FonctionTimer.c                          0x00000000   Number         0  fonctiontimer.o ABSOLUTE
    FonctionTimer.c                          0x00000000   Number         0  fonctiontimer.o ABSOLUTE
    Initialisation.c                         0x00000000   Number         0  initialisation.o ABSOLUTE
    Initialisation.c                         0x00000000   Number         0  initialisation.o ABSOLUTE
    Principale.asm                           0x00000000   Number         0  principale.o ABSOLUTE
    RTE\Device\STM32F103RB\startup_stm32f10x_md.s 0x00000000   Number         0  startup_stm32f10x_md.o ABSOLUTE
    RTE\Device\STM32F103RB\system_stm32f10x.c 0x00000000   Number         0  system_stm32f10x.o ABSOLUTE
    RTE\\Device\\STM32F103RB\\system_stm32f10x.c 0x00000000   Number         0  system_stm32f10x.o ABSOLUTE
    Spi.c                                    0x00000000   Number         0  spi.o ABSOLUTE
    Spi.c                                    0x00000000   Number         0  spi.o ABSOLUTE
    Warning.c                                0x00000000   Number         0  warning.o ABSOLUTE
    cdcmple.s                                0x00000000   Number         0  cdcmple.o ABSOLUTE
    cdrcmple.s                               0x00000000   Number         0  cdrcmple.o ABSOLUTE
    dc.s                                     0x00000000   Number         0  dc.o ABSOLUTE
    handlers.s                               0x00000000   Number         0  handlers.o ABSOLUTE
    init.s                                   0x00000000   Number         0  init.o ABSOLUTE
    RESET                                    0x08000000   Section      236  startup_stm32f10x_md.o(RESET)
    .ARM.Collect$$$$00000000                 0x080000ec   Section        0  entry.o(.ARM.Collect$$$$00000000)
    .ARM.Collect$$$$00000001                 0x080000ec   Section        4  entry2.o(.ARM.Collect$$$$00000001)
    .ARM.Collect$$$$00000004                 0x080000f0   Section        4  entry5.o(.ARM.Collect$$$$00000004)
    .ARM.Collect$$$$00000008                 0x080000f4   Section        0  entry7b.o(.ARM.Collect$$$$00000008)
    .ARM.Collect$$$$0000000A                 0x080000f4   Section        0  entry8b.o(.ARM.Collect$$$$0000000A)
    .ARM.Collect$$$$0000000B                 0x080000f4   Section        8  entry9a.o(.ARM.Collect$$$$0000000B)
    .ARM.Collect$$$$0000000D                 0x080000fc   Section        0  entry10a.o(.ARM.Collect$$$$0000000D)
    .ARM.Collect$$$$0000000F                 0x080000fc   Section        0  entry11a.o(.ARM.Collect$$$$0000000F)
    .ARM.Collect$$$$00002712                 0x080000fc   Section        4  entry2.o(.ARM.Collect$$$$00002712)
    __lit__00000000                          0x080000fc   Data           4  entry2.o(.ARM.Collect$$$$00002712)
    .text                                    0x08000100   Section       36  startup_stm32f10x_md.o(.text)
    .text                                    0x08000124   Section        0  fmul.o(.text)
    .text                                    0x08000188   Section        0  fdiv.o(.text)
    .text                                    0x08000204   Section        0  dmul.o(.text)
    .text                                    0x080002e8   Section        0  ddiv.o(.text)
    .text                                    0x080003c6   Section        0  ffltui.o(.text)
    .text                                    0x080003d0   Section        0  ffixui.o(.text)
    .text                                    0x080003f8   Section        0  f2d.o(.text)
    .text                                    0x08000420   Section       48  cdcmple.o(.text)
    .text                                    0x08000450   Section       48  cdrcmple.o(.text)
    .text                                    0x08000480   Section        0  d2f.o(.text)
    .text                                    0x080004b8   Section        0  iusefp.o(.text)
    .text                                    0x080004b8   Section        0  fepilogue.o(.text)
    .text                                    0x08000526   Section        0  depilogue.o(.text)
    .text                                    0x080005e0   Section       36  init.o(.text)
    .text                                    0x08000604   Section        0  llshl.o(.text)
    .text                                    0x08000622   Section        0  llushr.o(.text)
    i.Anim                                   0x08000644   Section        0  fonctiontimer.o(i.Anim)
    i.Config_SPI                             0x0800066c   Section        0  spi.o(i.Config_SPI)
    i.DMA1_Channel1_Event                    0x080006b0   Section        0  dma_stm32f10x.o(i.DMA1_Channel1_Event)
    i.DMA1_Channel1_IRQHandler               0x080006b4   Section        0  dma_stm32f10x.o(i.DMA1_Channel1_IRQHandler)
    i.DMA1_Channel2_Event                    0x080006d0   Section        0  dma_stm32f10x.o(i.DMA1_Channel2_Event)
    i.DMA1_Channel2_IRQHandler               0x080006d4   Section        0  dma_stm32f10x.o(i.DMA1_Channel2_IRQHandler)
    i.DMA1_Channel3_Event                    0x080006f0   Section        0  dma_stm32f10x.o(i.DMA1_Channel3_Event)
    i.DMA1_Channel3_IRQHandler               0x080006f4   Section        0  dma_stm32f10x.o(i.DMA1_Channel3_IRQHandler)
    i.DMA1_Channel4_Event                    0x08000710   Section        0  dma_stm32f10x.o(i.DMA1_Channel4_Event)
    i.DMA1_Channel4_IRQHandler               0x08000714   Section        0  dma_stm32f10x.o(i.DMA1_Channel4_IRQHandler)
    i.DMA1_Channel5_Event                    0x08000730   Section        0  dma_stm32f10x.o(i.DMA1_Channel5_Event)
    i.DMA1_Channel5_IRQHandler               0x08000734   Section        0  dma_stm32f10x.o(i.DMA1_Channel5_IRQHandler)
    i.DMA1_Channel6_Event                    0x08000750   Section        0  dma_stm32f10x.o(i.DMA1_Channel6_Event)
    i.DMA1_Channel6_IRQHandler               0x08000754   Section        0  dma_stm32f10x.o(i.DMA1_Channel6_IRQHandler)
    i.DMA1_Channel7_Event                    0x08000770   Section        0  dma_stm32f10x.o(i.DMA1_Channel7_Event)
    i.DMA1_Channel7_IRQHandler               0x08000774   Section        0  dma_stm32f10x.o(i.DMA1_Channel7_IRQHandler)
    i.GPIO_Configure                         0x08000790   Section        0  pilote_io_1.o(i.GPIO_Configure)
    i.Init_Cible                             0x080008dc   Section        0  initialisation.o(i.Init_Cible)
    i.Init_Dot                               0x080009e8   Section        0  initialisation.o(i.Init_Dot)
    i.Init_Port                              0x08000a60   Section        0  initialisation.o(i.Init_Port)
    i.Init_Timer1                            0x08000af0   Section        0  initialisation.o(i.Init_Timer1)
    i.Init_Timer2_PWM                        0x08000c64   Section        0  initialisation.o(i.Init_Timer2_PWM)
    i.Init_Timer3_Slave                      0x08000d80   Section        0  initialisation.o(i.Init_Timer3_Slave)
    i.Init_Timer4                            0x08000df0   Section        0  initialisation.o(i.Init_Timer4)
    i.Port_IO_Reset                          0x08000e64   Section        0  pilote_io_1.o(i.Port_IO_Reset)
    i.Port_IO_Set                            0x08000e74   Section        0  pilote_io_1.o(i.Port_IO_Set)
    i.SPI_Cmd                                0x08000e84   Section        0  stm32f10x_spi.o(i.SPI_Cmd)
    i.SPI_I2S_GetFlagStatus                  0x08000e9c   Section        0  stm32f10x_spi.o(i.SPI_I2S_GetFlagStatus)
    i.SPI_I2S_SendData16                     0x08000eae   Section        0  spi.o(i.SPI_I2S_SendData16)
    i.SPI_Init                               0x08000eb2   Section        0  stm32f10x_spi.o(i.SPI_Init)
    i.SendSPI                                0x08000ef0   Section        0  spi.o(i.SendSPI)
    i.SetSysClock                            0x08000f78   Section        0  system_stm32f10x.o(i.SetSysClock)
    SetSysClock                              0x08000f79   Thumb Code     8  system_stm32f10x.o(i.SetSysClock)
    i.SetSysClockTo72                        0x08000f80   Section        0  system_stm32f10x.o(i.SetSysClockTo72)
    SetSysClockTo72                          0x08000f81   Thumb Code   214  system_stm32f10x.o(i.SetSysClockTo72)
    i.SysTick_Handler                        0x08001060   Section        0  timer_systick_1.o(i.SysTick_Handler)
    i.SystemInit                             0x08001070   Section        0  system_stm32f10x.o(i.SystemInit)
    i.Systick_Period                         0x080010d0   Section        0  timer_systick_1.o(i.Systick_Period)
    i.Systick_Prio_IT                        0x080011e0   Section        0  timer_systick_1.o(i.Systick_Prio_IT)
    i.TIM1_CC_IRQHandler                     0x08001204   Section        0  fonctiontimer.o(i.TIM1_CC_IRQHandler)
    i.TIM1_UP_IRQHandler                     0x080012b8   Section        0  fonctiontimer.o(i.TIM1_UP_IRQHandler)
    i.TIM2_IRQHandler                        0x0800135c   Section        0  fonctiontimer.o(i.TIM2_IRQHandler)
    i.TIM3_IRQHandler                        0x08001360   Section        0  fonctiontimer.o(i.TIM3_IRQHandler)
    i.TIM4_IRQHandler                        0x080013b0   Section        0  fonctiontimer.o(i.TIM4_IRQHandler)
    i.__scatterload_copy                     0x08001424   Section       14  handlers.o(i.__scatterload_copy)
    i.__scatterload_null                     0x08001432   Section        2  handlers.o(i.__scatterload_null)
    i.__scatterload_zeroinit                 0x08001434   Section       14  handlers.o(i.__scatterload_zeroinit)
    moncode                                  0x08001444   Section       10  principale.o(moncode)
    moncode                                  0x08001450   Section      200  foncasm.o(moncode)
    .data                                    0x20000000   Section       19  initialisation.o(.data)
    .data                                    0x20000014   Section       24  fonctiontimer.o(.data)
    incre                                    0x20000024   Data           4  fonctiontimer.o(.data)
    Compteur                                 0x20000028   Data           4  fonctiontimer.o(.data)
    .data                                    0x2000002c   Section       96  warning.o(.data)
    .data                                    0x2000008c   Section        4  timer_systick_1.o(.data)
    Ptr_Systick                              0x2000008c   Data           4  timer_systick_1.o(.data)
    .bss                                     0x20000090   Section       18  spi.o(.bss)
    STACK                                    0x200000a8   Section     1024  startup_stm32f10x_md.o(STACK)

    Global Symbols

    Symbol Name                              Value     Ov Type        Size  Object(Section)

    BuildAttributes$$THM_ISAv4$P$D$K$B$S$PE$A:L22UL41UL21$X:L11$S22US41US21$IEEE1$IW$USESV6$~STKCKD$USESV7$~SHL$OTIME$ROPI$EBA8$MICROLIB$REQ8$PRES8$EABIv2 0x00000000   Number         0  anon$$obj.o ABSOLUTE
    __cpp_initialize__aeabi_                  - Undefined Weak Reference
    __cxa_finalize                            - Undefined Weak Reference
    __decompress                              - Undefined Weak Reference
    _clock_init                               - Undefined Weak Reference
    _microlib_exit                            - Undefined Weak Reference
    __Vectors_Size                           0x000000ec   Number         0  startup_stm32f10x_md.o ABSOLUTE
    __Vectors                                0x08000000   Data           4  startup_stm32f10x_md.o(RESET)
    __Vectors_End                            0x080000ec   Data           0  startup_stm32f10x_md.o(RESET)
    __main                                   0x080000ed   Thumb Code     0  entry.o(.ARM.Collect$$$$00000000)
    _main_stk                                0x080000ed   Thumb Code     0  entry2.o(.ARM.Collect$$$$00000001)
    _main_scatterload                        0x080000f1   Thumb Code     0  entry5.o(.ARM.Collect$$$$00000004)
    __main_after_scatterload                 0x080000f5   Thumb Code     0  entry5.o(.ARM.Collect$$$$00000004)
    _main_clock                              0x080000f5   Thumb Code     0  entry7b.o(.ARM.Collect$$$$00000008)
    _main_cpp_init                           0x080000f5   Thumb Code     0  entry8b.o(.ARM.Collect$$$$0000000A)
    _main_init                               0x080000f5   Thumb Code     0  entry9a.o(.ARM.Collect$$$$0000000B)
    __rt_final_cpp                           0x080000fd   Thumb Code     0  entry10a.o(.ARM.Collect$$$$0000000D)
    __rt_final_exit                          0x080000fd   Thumb Code     0  entry11a.o(.ARM.Collect$$$$0000000F)
    Reset_Handler                            0x08000101   Thumb Code     8  startup_stm32f10x_md.o(.text)
    NMI_Handler                              0x08000109   Thumb Code     2  startup_stm32f10x_md.o(.text)
    HardFault_Handler                        0x0800010b   Thumb Code     2  startup_stm32f10x_md.o(.text)
    MemManage_Handler                        0x0800010d   Thumb Code     2  startup_stm32f10x_md.o(.text)
    BusFault_Handler                         0x0800010f   Thumb Code     2  startup_stm32f10x_md.o(.text)
    UsageFault_Handler                       0x08000111   Thumb Code     2  startup_stm32f10x_md.o(.text)
    SVC_Handler                              0x08000113   Thumb Code     2  startup_stm32f10x_md.o(.text)
    DebugMon_Handler                         0x08000115   Thumb Code     2  startup_stm32f10x_md.o(.text)
    PendSV_Handler                           0x08000117   Thumb Code     2  startup_stm32f10x_md.o(.text)
    ADC1_2_IRQHandler                        0x0800011b   Thumb Code     0  startup_stm32f10x_md.o(.text)
    CAN1_RX1_IRQHandler                      0x0800011b   Thumb Code     0  startup_stm32f10x_md.o(.text)
    CAN1_SCE_IRQHandler                      0x0800011b   Thumb Code     0  startup_stm32f10x_md.o(.text)
    EXTI0_IRQHandler                         0x0800011b   Thumb Code     0  startup_stm32f10x_md.o(.text)
    EXTI15_10_IRQHandler                     0x0800011b   Thumb Code     0  startup_stm32f10x_md.o(.text)
    EXTI1_IRQHandler                         0x0800011b   Thumb Code     0  startup_stm32f10x_md.o(.text)
    EXTI2_IRQHandler                         0x0800011b   Thumb Code     0  startup_stm32f10x_md.o(.text)
    EXTI3_IRQHandler                         0x0800011b   Thumb Code     0  startup_stm32f10x_md.o(.text)
    EXTI4_IRQHandler                         0x0800011b   Thumb Code     0  startup_stm32f10x_md.o(.text)
    EXTI9_5_IRQHandler                       0x0800011b   Thumb Code     0  startup_stm32f10x_md.o(.text)
    FLASH_IRQHandler                         0x0800011b   Thumb Code     0  startup_stm32f10x_md.o(.text)
    I2C1_ER_IRQHandler                       0x0800011b   Thumb Code     0  startup_stm32f10x_md.o(.text)
    I2C1_EV_IRQHandler                       0x0800011b   Thumb Code     0  startup_stm32f10x_md.o(.text)
    I2C2_ER_IRQHandler                       0x0800011b   Thumb Code     0  startup_stm32f10x_md.o(.text)
    I2C2_EV_IRQHandler                       0x0800011b   Thumb Code     0  startup_stm32f10x_md.o(.text)
    PVD_IRQHandler                           0x0800011b   Thumb Code     0  startup_stm32f10x_md.o(.text)
    RCC_IRQHandler                           0x0800011b   Thumb Code     0  startup_stm32f10x_md.o(.text)
    RTCAlarm_IRQHandler                      0x0800011b   Thumb Code     0  startup_stm32f10x_md.o(.text)
    RTC_IRQHandler                           0x0800011b   Thumb Code     0  startup_stm32f10x_md.o(.text)
    SPI1_IRQHandler                          0x0800011b   Thumb Code     0  startup_stm32f10x_md.o(.text)
    SPI2_IRQHandler                          0x0800011b   Thumb Code     0  startup_stm32f10x_md.o(.text)
    TAMPER_IRQHandler                        0x0800011b   Thumb Code     0  startup_stm32f10x_md.o(.text)
    TIM1_BRK_IRQHandler                      0x0800011b   Thumb Code     0  startup_stm32f10x_md.o(.text)
    TIM1_TRG_COM_IRQHandler                  0x0800011b   Thumb Code     0  startup_stm32f10x_md.o(.text)
    USART1_IRQHandler                        0x0800011b   Thumb Code     0  startup_stm32f10x_md.o(.text)
    USART2_IRQHandler                        0x0800011b   Thumb Code     0  startup_stm32f10x_md.o(.text)
    USART3_IRQHandler                        0x0800011b   Thumb Code     0  startup_stm32f10x_md.o(.text)
    USBWakeUp_IRQHandler                     0x0800011b   Thumb Code     0  startup_stm32f10x_md.o(.text)
    USB_HP_CAN1_TX_IRQHandler                0x0800011b   Thumb Code     0  startup_stm32f10x_md.o(.text)
    USB_LP_CAN1_RX0_IRQHandler               0x0800011b   Thumb Code     0  startup_stm32f10x_md.o(.text)
    WWDG_IRQHandler                          0x0800011b   Thumb Code     0  startup_stm32f10x_md.o(.text)
    __aeabi_fmul                             0x08000125   Thumb Code   100  fmul.o(.text)
    __aeabi_fdiv                             0x08000189   Thumb Code   124  fdiv.o(.text)
    __aeabi_dmul                             0x08000205   Thumb Code   228  dmul.o(.text)
    __aeabi_ddiv                             0x080002e9   Thumb Code   222  ddiv.o(.text)
    __aeabi_ui2f                             0x080003c7   Thumb Code    10  ffltui.o(.text)
    __aeabi_f2uiz                            0x080003d1   Thumb Code    40  ffixui.o(.text)
    __aeabi_f2d                              0x080003f9   Thumb Code    38  f2d.o(.text)
    __aeabi_cdcmpeq                          0x08000421   Thumb Code     0  cdcmple.o(.text)
    __aeabi_cdcmple                          0x08000421   Thumb Code    48  cdcmple.o(.text)
    __aeabi_cdrcmple                         0x08000451   Thumb Code    48  cdrcmple.o(.text)
    __aeabi_d2f                              0x08000481   Thumb Code    56  d2f.o(.text)
    __I$use$fp                               0x080004b9   Thumb Code     0  iusefp.o(.text)
    _float_round                             0x080004b9   Thumb Code    18  fepilogue.o(.text)
    _float_epilogue                          0x080004cb   Thumb Code    92  fepilogue.o(.text)
    _double_round                            0x08000527   Thumb Code    30  depilogue.o(.text)
    _double_epilogue                         0x08000545   Thumb Code   156  depilogue.o(.text)
    __scatterload                            0x080005e1   Thumb Code    28  init.o(.text)
    __scatterload_rt2                        0x080005e1   Thumb Code     0  init.o(.text)
    __aeabi_llsl                             0x08000605   Thumb Code    30  llshl.o(.text)
    _ll_shift_l                              0x08000605   Thumb Code     0  llshl.o(.text)
    __aeabi_llsr                             0x08000623   Thumb Code    32  llushr.o(.text)
    _ll_ushift_r                             0x08000623   Thumb Code     0  llushr.o(.text)
    Anim                                     0x08000645   Thumb Code    32  fonctiontimer.o(i.Anim)
    Config_SPI                               0x0800066d   Thumb Code    58  spi.o(i.Config_SPI)
    DMA1_Channel1_Event                      0x080006b1   Thumb Code     2  dma_stm32f10x.o(i.DMA1_Channel1_Event)
    DMA1_Channel1_IRQHandler                 0x080006b5   Thumb Code    22  dma_stm32f10x.o(i.DMA1_Channel1_IRQHandler)
    DMA1_Channel2_Event                      0x080006d1   Thumb Code     2  dma_stm32f10x.o(i.DMA1_Channel2_Event)
    DMA1_Channel2_IRQHandler                 0x080006d5   Thumb Code    24  dma_stm32f10x.o(i.DMA1_Channel2_IRQHandler)
    DMA1_Channel3_Event                      0x080006f1   Thumb Code     2  dma_stm32f10x.o(i.DMA1_Channel3_Event)
    DMA1_Channel3_IRQHandler                 0x080006f5   Thumb Code    24  dma_stm32f10x.o(i.DMA1_Channel3_IRQHandler)
    DMA1_Channel4_Event                      0x08000711   Thumb Code     2  dma_stm32f10x.o(i.DMA1_Channel4_Event)
    DMA1_Channel4_IRQHandler                 0x08000715   Thumb Code    24  dma_stm32f10x.o(i.DMA1_Channel4_IRQHandler)
    DMA1_Channel5_Event                      0x08000731   Thumb Code     2  dma_stm32f10x.o(i.DMA1_Channel5_Event)
    DMA1_Channel5_IRQHandler                 0x08000735   Thumb Code    24  dma_stm32f10x.o(i.DMA1_Channel5_IRQHandler)
    DMA1_Channel6_Event                      0x08000751   Thumb Code     2  dma_stm32f10x.o(i.DMA1_Channel6_Event)
    DMA1_Channel6_IRQHandler                 0x08000755   Thumb Code    24  dma_stm32f10x.o(i.DMA1_Channel6_IRQHandler)
    DMA1_Channel7_Event                      0x08000771   Thumb Code     2  dma_stm32f10x.o(i.DMA1_Channel7_Event)
    DMA1_Channel7_IRQHandler                 0x08000775   Thumb Code    24  dma_stm32f10x.o(i.DMA1_Channel7_IRQHandler)
    GPIO_Configure                           0x08000791   Thumb Code   314  pilote_io_1.o(i.GPIO_Configure)
    Init_Cible                               0x080008dd   Thumb Code   218  initialisation.o(i.Init_Cible)
    Init_Dot                                 0x080009e9   Thumb Code   112  initialisation.o(i.Init_Dot)
    Init_Port                                0x08000a61   Thumb Code   134  initialisation.o(i.Init_Port)
    Init_Timer1                              0x08000af1   Thumb Code   336  initialisation.o(i.Init_Timer1)
    Init_Timer2_PWM                          0x08000c65   Thumb Code   262  initialisation.o(i.Init_Timer2_PWM)
    Init_Timer3_Slave                        0x08000d81   Thumb Code    94  initialisation.o(i.Init_Timer3_Slave)
    Init_Timer4                              0x08000df1   Thumb Code   100  initialisation.o(i.Init_Timer4)
    Port_IO_Reset                            0x08000e65   Thumb Code    16  pilote_io_1.o(i.Port_IO_Reset)
    Port_IO_Set                              0x08000e75   Thumb Code    16  pilote_io_1.o(i.Port_IO_Set)
    SPI_Cmd                                  0x08000e85   Thumb Code    24  stm32f10x_spi.o(i.SPI_Cmd)
    SPI_I2S_GetFlagStatus                    0x08000e9d   Thumb Code    18  stm32f10x_spi.o(i.SPI_I2S_GetFlagStatus)
    SPI_I2S_SendData16                       0x08000eaf   Thumb Code     4  spi.o(i.SPI_I2S_SendData16)
    SPI_Init                                 0x08000eb3   Thumb Code    60  stm32f10x_spi.o(i.SPI_Init)
    SendSPI                                  0x08000ef1   Thumb Code   130  spi.o(i.SendSPI)
    SysTick_Handler                          0x08001061   Thumb Code    10  timer_systick_1.o(i.SysTick_Handler)
    SystemInit                               0x08001071   Thumb Code    78  system_stm32f10x.o(i.SystemInit)
    Systick_Period                           0x080010d1   Thumb Code   256  timer_systick_1.o(i.Systick_Period)
    Systick_Prio_IT                          0x080011e1   Thumb Code    28  timer_systick_1.o(i.Systick_Prio_IT)
    TIM1_CC_IRQHandler                       0x08001205   Thumb Code   158  fonctiontimer.o(i.TIM1_CC_IRQHandler)
    TIM1_UP_IRQHandler                       0x080012b9   Thumb Code   130  fonctiontimer.o(i.TIM1_UP_IRQHandler)
    TIM2_IRQHandler                          0x0800135d   Thumb Code     4  fonctiontimer.o(i.TIM2_IRQHandler)
    TIM3_IRQHandler                          0x08001361   Thumb Code    68  fonctiontimer.o(i.TIM3_IRQHandler)
    TIM4_IRQHandler                          0x080013b1   Thumb Code    90  fonctiontimer.o(i.TIM4_IRQHandler)
    __scatterload_copy                       0x08001425   Thumb Code    14  handlers.o(i.__scatterload_copy)
    __scatterload_null                       0x08001433   Thumb Code     2  handlers.o(i.__scatterload_null)
    __scatterload_zeroinit                   0x08001435   Thumb Code    14  handlers.o(i.__scatterload_zeroinit)
    main                                     0x08001445   Thumb Code    10  principale.o(moncode)
    Envoie192Boucle                          0x08001451   Thumb Code   108  foncasm.o(moncode)
    Envoie96Dot                              0x080014bd   Thumb Code    78  foncasm.o(moncode)
    Region$$Table$$Base                      0x08001518   Number         0  anon$$obj.o(Region$$Table)
    Region$$Table$$Limit                     0x08001538   Number         0  anon$$obj.o(Region$$Table)
    PrtSurImage                              0x20000000   Data           4  initialisation.o(.data)
    BarretEnCours                            0x20000004   Data           4  initialisation.o(.data)
    DataSend                                 0x20000008   Data           1  initialisation.o(.data)
    Angle                                    0x2000000c   Data           4  initialisation.o(.data)
    CinqDots                                 0x20000010   Data           3  initialisation.o(.data)
    VitesseSuffisante                        0x20000014   Data           4  fonctiontimer.o(.data)
    SecteurEnCours                           0x20000018   Data           4  fonctiontimer.o(.data)
    ImageEnCours                             0x2000001c   Data           4  fonctiontimer.o(.data)
    increment                                0x20000020   Data           4  fonctiontimer.o(.data)
    warning                                  0x2000002c   Data          96  warning.o(.data)
    SPI_InitStructure                        0x20000090   Data          18  spi.o(.bss)
    __initial_sp                             0x200004a8   Data           0  startup_stm32f10x_md.o(STACK)



==============================================================================

Memory Map of the image

  Image Entry point : 0x080000ed

  Load Region LR_IROM1 (Base: 0x08000000, Size: 0x000015c8, Max: 0x00020000, ABSOLUTE)

    Execution Region ER_IROM1 (Exec base: 0x08000000, Load base: 0x08000000, Size: 0x00001538, Max: 0x00020000, ABSOLUTE)

    Exec Addr    Load Addr    Size         Type   Attr      Idx    E Section Name        Object

    0x08000000   0x08000000   0x000000ec   Data   RO         1219    RESET               startup_stm32f10x_md.o
    0x080000ec   0x080000ec   0x00000000   Code   RO         1643  * .ARM.Collect$$$$00000000  mc_w.l(entry.o)
    0x080000ec   0x080000ec   0x00000004   Code   RO         1666    .ARM.Collect$$$$00000001  mc_w.l(entry2.o)
    0x080000f0   0x080000f0   0x00000004   Code   RO         1669    .ARM.Collect$$$$00000004  mc_w.l(entry5.o)
    0x080000f4   0x080000f4   0x00000000   Code   RO         1671    .ARM.Collect$$$$00000008  mc_w.l(entry7b.o)
    0x080000f4   0x080000f4   0x00000000   Code   RO         1673    .ARM.Collect$$$$0000000A  mc_w.l(entry8b.o)
    0x080000f4   0x080000f4   0x00000008   Code   RO         1674    .ARM.Collect$$$$0000000B  mc_w.l(entry9a.o)
    0x080000fc   0x080000fc   0x00000000   Code   RO         1676    .ARM.Collect$$$$0000000D  mc_w.l(entry10a.o)
    0x080000fc   0x080000fc   0x00000000   Code   RO         1678    .ARM.Collect$$$$0000000F  mc_w.l(entry11a.o)
    0x080000fc   0x080000fc   0x00000004   Code   RO         1667    .ARM.Collect$$$$00002712  mc_w.l(entry2.o)
    0x08000100   0x08000100   0x00000024   Code   RO         1220    .text               startup_stm32f10x_md.o
    0x08000124   0x08000124   0x00000064   Code   RO         1646    .text               mf_w.l(fmul.o)
    0x08000188   0x08000188   0x0000007c   Code   RO         1648    .text               mf_w.l(fdiv.o)
    0x08000204   0x08000204   0x000000e4   Code   RO         1650    .text               mf_w.l(dmul.o)
    0x080002e8   0x080002e8   0x000000de   Code   RO         1652    .text               mf_w.l(ddiv.o)
    0x080003c6   0x080003c6   0x0000000a   Code   RO         1654    .text               mf_w.l(ffltui.o)
    0x080003d0   0x080003d0   0x00000028   Code   RO         1656    .text               mf_w.l(ffixui.o)
    0x080003f8   0x080003f8   0x00000026   Code   RO         1658    .text               mf_w.l(f2d.o)
    0x0800041e   0x0800041e   0x00000002   PAD
    0x08000420   0x08000420   0x00000030   Code   RO         1660    .text               mf_w.l(cdcmple.o)
    0x08000450   0x08000450   0x00000030   Code   RO         1662    .text               mf_w.l(cdrcmple.o)
    0x08000480   0x08000480   0x00000038   Code   RO         1664    .text               mf_w.l(d2f.o)
    0x080004b8   0x080004b8   0x00000000   Code   RO         1680    .text               mc_w.l(iusefp.o)
    0x080004b8   0x080004b8   0x0000006e   Code   RO         1681    .text               mf_w.l(fepilogue.o)
    0x08000526   0x08000526   0x000000ba   Code   RO         1683    .text               mf_w.l(depilogue.o)
    0x080005e0   0x080005e0   0x00000024   Code   RO         1685    .text               mc_w.l(init.o)
    0x08000604   0x08000604   0x0000001e   Code   RO         1687    .text               mc_w.l(llshl.o)
    0x08000622   0x08000622   0x00000020   Code   RO         1689    .text               mc_w.l(llushr.o)
    0x08000642   0x08000642   0x00000002   PAD
    0x08000644   0x08000644   0x00000028   Code   RO         1380    i.Anim              Matos.lib(fonctiontimer.o)
    0x0800066c   0x0800066c   0x00000044   Code   RO         1489    i.Config_SPI        Matos.lib(spi.o)
    0x080006b0   0x080006b0   0x00000002   Code   RO         1028    i.DMA1_Channel1_Event  dma_stm32f10x.o
    0x080006b2   0x080006b2   0x00000002   PAD
    0x080006b4   0x080006b4   0x0000001c   Code   RO         1029    i.DMA1_Channel1_IRQHandler  dma_stm32f10x.o
    0x080006d0   0x080006d0   0x00000002   Code   RO         1030    i.DMA1_Channel2_Event  dma_stm32f10x.o
    0x080006d2   0x080006d2   0x00000002   PAD
    0x080006d4   0x080006d4   0x0000001c   Code   RO         1031    i.DMA1_Channel2_IRQHandler  dma_stm32f10x.o
    0x080006f0   0x080006f0   0x00000002   Code   RO         1032    i.DMA1_Channel3_Event  dma_stm32f10x.o
    0x080006f2   0x080006f2   0x00000002   PAD
    0x080006f4   0x080006f4   0x0000001c   Code   RO         1033    i.DMA1_Channel3_IRQHandler  dma_stm32f10x.o
    0x08000710   0x08000710   0x00000002   Code   RO         1034    i.DMA1_Channel4_Event  dma_stm32f10x.o
    0x08000712   0x08000712   0x00000002   PAD
    0x08000714   0x08000714   0x0000001c   Code   RO         1035    i.DMA1_Channel4_IRQHandler  dma_stm32f10x.o
    0x08000730   0x08000730   0x00000002   Code   RO         1036    i.DMA1_Channel5_Event  dma_stm32f10x.o
    0x08000732   0x08000732   0x00000002   PAD
    0x08000734   0x08000734   0x0000001c   Code   RO         1037    i.DMA1_Channel5_IRQHandler  dma_stm32f10x.o
    0x08000750   0x08000750   0x00000002   Code   RO         1038    i.DMA1_Channel6_Event  dma_stm32f10x.o
    0x08000752   0x08000752   0x00000002   PAD
    0x08000754   0x08000754   0x0000001c   Code   RO         1039    i.DMA1_Channel6_IRQHandler  dma_stm32f10x.o
    0x08000770   0x08000770   0x00000002   Code   RO         1040    i.DMA1_Channel7_Event  dma_stm32f10x.o
    0x08000772   0x08000772   0x00000002   PAD
    0x08000774   0x08000774   0x0000001c   Code   RO         1041    i.DMA1_Channel7_IRQHandler  dma_stm32f10x.o
    0x08000790   0x08000790   0x0000014c   Code   RO         1542    i.GPIO_Configure    Matos.lib(pilote_io_1.o)
    0x080008dc   0x080008dc   0x0000010c   Code   RO         1273    i.Init_Cible        Matos.lib(initialisation.o)
    0x080009e8   0x080009e8   0x00000078   Code   RO         1274    i.Init_Dot          Matos.lib(initialisation.o)
    0x08000a60   0x08000a60   0x00000090   Code   RO         1275    i.Init_Port         Matos.lib(initialisation.o)
    0x08000af0   0x08000af0   0x00000174   Code   RO         1277    i.Init_Timer1       Matos.lib(initialisation.o)
    0x08000c64   0x08000c64   0x0000011c   Code   RO         1278    i.Init_Timer2_PWM   Matos.lib(initialisation.o)
    0x08000d80   0x08000d80   0x00000070   Code   RO         1279    i.Init_Timer3_Slave  Matos.lib(initialisation.o)
    0x08000df0   0x08000df0   0x00000074   Code   RO         1280    i.Init_Timer4       Matos.lib(initialisation.o)
    0x08000e64   0x08000e64   0x00000010   Code   RO         1548    i.Port_IO_Reset     Matos.lib(pilote_io_1.o)
    0x08000e74   0x08000e74   0x00000010   Code   RO         1549    i.Port_IO_Set       Matos.lib(pilote_io_1.o)
    0x08000e84   0x08000e84   0x00000018   Code   RO          317    i.SPI_Cmd           stm32f10x_spi.o
    0x08000e9c   0x08000e9c   0x00000012   Code   RO          325    i.SPI_I2S_GetFlagStatus  stm32f10x_spi.o
    0x08000eae   0x08000eae   0x00000004   Code   RO         1490    i.SPI_I2S_SendData16  Matos.lib(spi.o)
    0x08000eb2   0x08000eb2   0x0000003c   Code   RO          330    i.SPI_Init          stm32f10x_spi.o
    0x08000eee   0x08000eee   0x00000002   PAD
    0x08000ef0   0x08000ef0   0x00000088   Code   RO         1491    i.SendSPI           Matos.lib(spi.o)
    0x08000f78   0x08000f78   0x00000008   Code   RO         1227    i.SetSysClock       system_stm32f10x.o
    0x08000f80   0x08000f80   0x000000e0   Code   RO         1228    i.SetSysClockTo72   system_stm32f10x.o
    0x08001060   0x08001060   0x00000010   Code   RO         1608    i.SysTick_Handler   Matos.lib(timer_systick_1.o)
    0x08001070   0x08001070   0x00000060   Code   RO         1230    i.SystemInit        system_stm32f10x.o
    0x080010d0   0x080010d0   0x00000110   Code   RO         1609    i.Systick_Period    Matos.lib(timer_systick_1.o)
    0x080011e0   0x080011e0   0x00000024   Code   RO         1610    i.Systick_Prio_IT   Matos.lib(timer_systick_1.o)
    0x08001204   0x08001204   0x000000b4   Code   RO         1389    i.TIM1_CC_IRQHandler  Matos.lib(fonctiontimer.o)
    0x080012b8   0x080012b8   0x000000a4   Code   RO         1390    i.TIM1_UP_IRQHandler  Matos.lib(fonctiontimer.o)
    0x0800135c   0x0800135c   0x00000004   Code   RO         1391    i.TIM2_IRQHandler   Matos.lib(fonctiontimer.o)
    0x08001360   0x08001360   0x00000050   Code   RO         1392    i.TIM3_IRQHandler   Matos.lib(fonctiontimer.o)
    0x080013b0   0x080013b0   0x00000074   Code   RO         1393    i.TIM4_IRQHandler   Matos.lib(fonctiontimer.o)
    0x08001424   0x08001424   0x0000000e   Code   RO         1693    i.__scatterload_copy  mc_w.l(handlers.o)
    0x08001432   0x08001432   0x00000002   Code   RO         1694    i.__scatterload_null  mc_w.l(handlers.o)
    0x08001434   0x08001434   0x0000000e   Code   RO         1695    i.__scatterload_zeroinit  mc_w.l(handlers.o)
    0x08001442   0x08001442   0x00000002   PAD
    0x08001444   0x08001444   0x0000000a   Code   RO            2    moncode             principale.o
    0x0800144e   0x0800144e   0x00000002   PAD
    0x08001450   0x08001450   0x000000c8   Code   RO         1535    moncode             Matos.lib(foncasm.o)
    0x08001518   0x08001518   0x00000020   Data   RO         1691    Region$$Table       anon$$obj.o


    Execution Region RW_IRAM1 (Exec base: 0x20000000, Load base: 0x08001538, Size: 0x000004a8, Max: 0x00005000, ABSOLUTE)

    Exec Addr    Load Addr    Size         Type   Attr      Idx    E Section Name        Object

    0x20000000   0x08001538   0x00000013   Data   RW         1281    .data               Matos.lib(initialisation.o)
    0x20000013   0x0800154b   0x00000001   PAD
    0x20000014   0x0800154c   0x00000018   Data   RW         1394    .data               Matos.lib(fonctiontimer.o)
    0x2000002c   0x08001564   0x00000060   Data   RW         1525    .data               Matos.lib(warning.o)
    0x2000008c   0x080015c4   0x00000004   Data   RW         1611    .data               Matos.lib(timer_systick_1.o)
    0x20000090        -       0x00000012   Zero   RW         1492    .bss                Matos.lib(spi.o)
    0x200000a2   0x080015c8   0x00000006   PAD
    0x200000a8        -       0x00000400   Zero   RW         1217    STACK               startup_stm32f10x_md.o


==============================================================================

Image component sizes


      Code (inc. data)   RO Data    RW Data    ZI Data      Debug   Object Name

       210         30          0          0          0       7259   dma_stm32f10x.o
         0          0          0          0          0     213380   misc.o
        10          0          0          0          0        400   principale.o
        36          8        236          0       1024        860   startup_stm32f10x_md.o
       102          0          0          0          0       2941   stm32f10x_spi.o
       328         28          0          0          0       2205   system_stm32f10x.o

    ----------------------------------------------------------------------
       704         66        268          0       1024     227045   Object Totals
         0          0         32          0          0          0   (incl. Generated)
        18          0          0          0          0          0   (incl. Padding)

    ----------------------------------------------------------------------

      Code (inc. data)   RO Data    RW Data    ZI Data      Debug   Library Member Name

       200         14          0          0          0        460   foncasm.o
       584        102          0         24          0       3477   fonctiontimer.o
      1416        160          0         19          0     225316   initialisation.o
       364         18          0          0          0       2487   pilote_io_1.o
       208         16          0          0         18       2436   spi.o
       324         30          0          4          0       2509   timer_systick_1.o
         0          0          0         96          0        582   warning.o
         0          0          0          0          0          0   entry.o
         0          0          0          0          0          0   entry10a.o
         0          0          0          0          0          0   entry11a.o
         8          4          0          0          0          0   entry2.o
         4          0          0          0          0          0   entry5.o
         0          0          0          0          0          0   entry7b.o
         0          0          0          0          0          0   entry8b.o
         8          4          0          0          0          0   entry9a.o
        30          0          0          0          0          0   handlers.o
        36          8          0          0          0         68   init.o
         0          0          0          0          0          0   iusefp.o
        30          0          0          0          0         68   llshl.o
        32          0          0          0          0         68   llushr.o
        48          0          0          0          0         68   cdcmple.o
        48          0          0          0          0         68   cdrcmple.o
        56          0          0          0          0         88   d2f.o
       222          0          0          0          0        100   ddiv.o
       186          0          0          0          0        176   depilogue.o
       228          0          0          0          0         96   dmul.o
        38          0          0          0          0         68   f2d.o
       124          0          0          0          0         88   fdiv.o
       110          0          0          0          0        168   fepilogue.o
        40          0          0          0          0         68   ffixui.o
        10          0          0          0          0         68   ffltui.o
       100          0          0          0          0         76   fmul.o

    ----------------------------------------------------------------------
      4460        356          0        144         24     238603   Library Totals
         6          0          0          1          6          0   (incl. Padding)

    ----------------------------------------------------------------------

      Code (inc. data)   RO Data    RW Data    ZI Data      Debug   Library Name

      3096        340          0        143         18     237267   Matos.lib
       148         16          0          0          0        204   mc_w.l
      1210          0          0          0          0       1132   mf_w.l

    ----------------------------------------------------------------------
      4460        356          0        144         24     238603   Library Totals

    ----------------------------------------------------------------------

==============================================================================


      Code (inc. data)   RO Data    RW Data    ZI Data      Debug   

      5164        422        268        144       1048     462992   Grand Totals
      5164        422        268        144       1048     462992   ELF Image Totals
      5164        422        268        144          0          0   ROM Totals

==============================================================================

    Total RO  Size (Code + RO Data)                 5432 (   5.30kB)
    Total RW  Size (RW Data + ZI Data)              1192 (   1.16kB)
    Total ROM Size (Code + RO Data + RW Data)       5576 (   5.45kB)

==============================================================================

